:020000021000EC
:10E000004BC0000066C0000064C0000062C0000099
:10E0100060C000005EC000005CC000005AC000008C
:10E0200058C0000056C00000BEC4000052C000002E
:10E0300050C000004EC000004CC000004AC00000AC
:10E0400048C0000046C0000044C0000042C00000BC
:10E0500041C000003EC000003CC000003AC00000CB
:10E0600038C0000036C0000034C0000032C00000DC
:10E0700030C000002EC000002CC000002AC00000EC
:10E0800028C0000026C0000024C0000022C00000FC
:10E0900020C000001EC0000011241FBECFEFD0E240
:10E0A000DEBFCDBF11E0A0E0B1E0E8EBFEEE01E0A5
:10E0B0000BBF02C007900D92AC38B107D9F711E041
:10E0C000ACE8B1E001C01D92AA39B107E1F734D341
:10E0D000F1C696CF1F920F920FB60F9211240F9098
:10E0E0000FBE0F901F90189584E08093E9000DC03B
:10E0F0008091E8008B778093E80003C08EB388237B
:10E1000051F08091E80082FFF9CF8091E80085FF0F
:10E11000EFCF8091F1000895982F83E08093E9007C
:10E120008091E80085FD0DC08091E8008E77809396
:10E13000E80003C08EB3882331F08091E80080FFAF
:10E14000F9CF9093F10008954F925F926F927F9272
:10E150008F929F92AF92BF92CF92DF92EF92FF92F7
:10E160000F931F93CF93DF9384E08093E900809116
:10E17000E80082FF73C2B8DF182F853419F41092BB
:10E18000080103C0843519F4AFDF8DE03DC28C3443
:10E19000E1F38035D1F3843711F484E495C08136FE
:10E1A00011F489E531C28134B1F49EDF182F9CDF70
:10E1B00090E0880F991FAA2797FDA095BA2F312FBD
:10E1C000330F20E0442737FD4095542F822B932BAB
:10E1D000A42BB52BEAC1803711F483E515C2833532
:10E1E00049F4C0E0D1E0899197DF41E0C730D4071E
:10E1F000D1F70BC2863521F481E38EDF80E304C2C0
:10E20000833731F482E888DF87E986DF8EE1FCC15D
:10E21000853629F580E090E0A0E0B0E033E025E02D
:10E22000FC01A0935B0030935700E89507B600FC13
:10E23000FDCFFC01A0935B0020935700E89507B643
:10E2400000FCFDCF80509F4FAF4FBF4F803040EE5E
:10E25000940741E0A40740E0B40711F796CF8C364D
:10E2600051F442DF809599E0E1E0F0E0082E9093D0
:10E270005700E8958ACF823739F4E1E0F0E089E091
:10E28000809357008491C0C1863439F4E0E0F0E017
:10E2900089E0809357008491B7C18E3439F4E3E06C
:10E2A000F0E089E0809357008491AEC1813539F464
:10E2B000E2E0F0E089E0809357008491A5C18236C6
:10E2C00031F489E529DF81E027DF80E09DC18234D8
:10E2D00019F0873609F0E6C007DF082F05DFF82EB2
:10E2E00003DF682E8554823008F08DC1902F80E0C6
:10E2F000CF2DD0E0C82BD92B173609F050C081E1C3
:10E3000080935700E895DD24CC24C39444C0E0906A
:10E310008C01F0908D0100918E0110918F0186E4A7
:10E32000681601F58D2D90E0A0E0B0E08E299F29C0
:10E33000A02BB12BABBFFC018791EEDEDD2081F07D
:10E3400082E090E0A0E0B0E0E80EF91E0A1F1B1F7B
:10E35000E0928C01F0928D0100938E0110938F0159
:10E36000DC2418C0D801C701B695A7959795879565
:10E370008BD5D2DE82E090E0A0E0B0E0E80EF91E9E
:10E380000A1F1B1FE0928C01F0928D0100938E01F9
:10E3900010938F012197209709F0B9CF36C1809053
:10E3A0008C0190908D01A0908E01B0908F0196E429
:10E3B000691609F061C083E0F401A0925B008093CC
:10E3C0005700E89507B600FCFDCF56C0A6E46A16D4
:10E3D00071F5772041F1E0908C01F0908D01009172
:10E3E0008E0110918F0180DED82ECC24852D90E0F7
:10E3F0008C299D290C01F70100935B004092570086
:10E40000E895112482E090E0A0E0B0E0E80EF91E6B
:10E410000A1F1B1FE0928C01F0928D0100938E0168
:10E4200010938F0102C060DE582E742423C0E09048
:10E430008C01F0908D0100918E0110918F01169545
:10E440000795F794E79450DE682FC70125D5809192
:10E450008C0190918D01A0918E01B0918F01029657
:10E46000A11DB11D80938C0190938D01A0938E010D
:10E47000B0938F01219704C05524772444244394FA
:10E48000209709F0A3CF96E4691609F07ECE85E0C7
:10E49000F401A0925B0080935700E89507B600FC5A
:10E4A000FDCF73CE8334A1F4E0908C01F0908D0108
:10E4B00000918E0110918F0117DE90E021E00C0198
:10E4C000F70100935B0020935700E89511245DCE7F
:10E4D000833639F5E0908C01F0908D0100918E012A
:10E4E00010918F0101DEA8019701216090E061E0A9
:10E4F0000C01F90140935B0060935700E8951124EB
:10E5000082E090E0A0E0B0E0E80EF91E0A1F1B1FB9
:10E51000E0928C01F0928D0100938E0110938F0197
:10E5200034CE8D3699F480918C0190918D01A0911B
:10E530008E01B0918F0125E0FC01A0935B00209338
:10E540005700E89507B600FCFDCF1FCE823581F459
:10E55000E0908C01F0908D0100918E0110918F015F
:10E560000BBFF701E790F6908F2DD6DD8E2D4CC0B6
:10E57000843421F5E0908C01F0908D0100918E01A2
:10E5800010918F0116950795F794E794ADDD682FEC
:10E59000C70182D480918C0190918D01A0918E0150
:10E5A000B0918F010296A11DB11D80938C019093B3
:10E5B0008D01A0938E01B0938F01E7CD843609F5CC
:10E5C000E0908C01F0908D0100918E0110918F01EF
:10E5D000D801C701B695A7959795879555D49CDD29
:10E5E00082E090E0A0E0B0E0E80EF91E0A1F1B1FD9
:10E5F000E0928C01F0928D0100938E0110938F01B7
:10E6000004C08B3111F08FE387DD83E08093E90054
:10E610009091E8008091E8008E778093E80095FF64
:10E6200004C010C08EB38823C9F08091E80080FF39
:10E63000F9CF8091E8008E778093E80003C08EB315
:10E64000882361F08091E80080FFF9CF84E0809317
:10E65000E9008091E8008B778093E800DF91CF910B
:10E660001F910F91FF90EF90DF90CF90BF90AF90F0
:10E670009F908F907F906F905F904F9008959091B2
:10E680009201892F8F77813249F5809193018032F1
:10E69000A1F0813219F5913A09F58091E800877F60
:10E6A0008093E80089E091E067E070E031D28091EA
:10E6B000E8008B778093E8000895913279F4809197
:10E6C000E800877F8093E80089E091E067E070E0F0
:10E6D0007BD28091E8008E778093E800089582E0F5
:10E6E00061EC42E0D4D083E061E842E1D0D084E044
:10E6F00060E842E1CCC01F9384B7877F84BF88E184
:10E700000FB6F89480936000109260000FBE90E006
:10E7100080E80FB6F89480936100909361000FBE7B
:10E7200011E015BF82E085BF28D110936F0083E010
:10E73000809381001F910895DF93CF9300D0CDB7D0
:10E74000DEB78091E0FF9091E1FF9A838983898110
:10E750009A81D1DF789402C0F7DC84D380910801DC
:10E760008823D1F78091E00081608093E0002CE065
:10E7700088E190E00FB6F894A895809360000FBEF2
:10E7800020936000FFCF9B01AC0107B600FCFDCFDA
:10E79000F999FECF83E0F90140935B008093570025
:10E7A000E89581E180935700E89508959B01AC01BD
:10E7B00007B600FCFDCFF999FECF85E0F901409343
:10E7C0005B0080935700E89581E180935700E895BE
:10E7D00008950F931F938B019C0107B600FCFDCF9A
:10E7E000F999FECF81E00A01F80120935B00809344
:10E7F0005700E89511241F910F91089521E2FC0123
:10E80000209357002491822F089529E0FC01209342
:10E8100057002491822F0895E1E0F0E089E0809391
:10E82000570084910895982F07B600FCFDCFF99901
:10E83000FECF909589E0E1E0F0E0092E809357004B
:10E84000E8950895FA01923071F0933089F0913093
:10E8500029F480E191E022E130E015C080E090E011
:10E8600020E030E010C082E291E02EE330E00BC007
:10E87000882329F480E691E024E030E004C084E6B7
:10E8800091E026E230E091838083C901089580936E
:10E89000E9008091EB0081608093EB001092ED0025
:10E8A0006093EC004093ED008091EE00881F882774
:10E8B000881F08958091920188238CF403C08EB341
:10E8C0008823B1F08091E80082FFF9CF8091E800C1
:10E8D0008B778093E80008958EB3882349F0809168
:10E8E000E80080FFF9CF8091E8008E778093E80000
:10E8F0000895EF92FF920F931F9348D04FD008EDE9
:10E9000010E0F80180818F77808380818068808328
:10E9100080818F7D8083E7EDF0E080818068808357
:10E9200019BC1EBA1092900180EEE82EF12CF7016E
:10E9300080818B7F8083F80180818160808380E08B
:10E9400060E042E0A4DFE1EEF0E080818E7F808332
:10E95000E2EEF0E080818160808380818860808346
:10E96000F70180818E7F8083F801808180618083C0
:10E970001F910F91FF90EF900895E7EDF0E08081F7
:10E980008160808381E080939101B3CFE8EDF0E076
:10E9900080818C7F80831092E20008951092DA00CB
:10E9A0001092E10008951F920F920FB60F920BB6CE
:10E9B0000F9211242F933F934F935F936F937F9305
:10E9C0008F939F93AF93BF93EF93FF938091DA0060
:10E9D00080FF1BC08091D80080FF17C08091DA00B3
:10E9E0008E7F8093DA008091D90080FF0BC084E194
:10E9F00089BD86E189BD09B400FEFDCF81E08EBBF3
:10EA000030D203C019BC1EBA2CD28091E10080FF25
:10EA100017C08091E20080FF13C08091E2008E7FDA
:10EA20008093E2008091E20080618093E200809117
:10EA3000D80080628093D80019BC85E08EBB11D2CB
:10EA40008091E10084FF2CC08091E20084FF28C007
:10EA500084E189BD86E189BD09B400FEFDCF8091C6
:10EA6000D8008F7D8093D8008091E1008F7E8093C5
:10EA7000E1008091E2008F7E8093E2008091E200CD
:10EA800081608093E20080919001882331F480912D
:10EA9000E30087FD02C081E001C084E08EBBE1D1CC
:10EAA0008091E10083FF21C08091E20083FF1DC0BF
:10EAB0008091E100877F8093E10082E08EBB10921D
:10EAC00090018091E1008E7F8093E1008091E200CF
:10EAD0008E7F8093E2008091E20080618093E2006B
:10EAE00080E060E042E0D3DEBCD1FF91EF91BF91C6
:10EAF000AF919F918F917F916F915F914F913F91D6
:10EB00002F910F900BBE0F900FBE0F901F90189576
:10EB10009C0140919801509199014617570718F4AC
:10EB2000F90190E03CC06115710511F0AB01F8CF1F
:10EB30008091E8008E778093E80040E050E0F0CFCD
:10EB40008EB38823E9F18530E9F18091E80083FFF5
:10EB500002C081E008958091E80082FD2BC0809181
:10EB6000E80080FF1CC02091F2003091F30007C044
:10EB700081918093F100415050402F5F3F4F4115EC
:10EB8000510519F02830310598F390E0283031050F
:10EB900009F491E08091E8008E778093E8004115B8
:10EBA000510571F6992361F605C08EB3882341F0B3
:10EBB000853041F08091E80082FFF7CF80E0089532
:10EBC00082E0089583E008959C016115710529F4A0
:10EBD0008091E8008B778093E800F90121C08EB323
:10EBE000882369F1853069F18091E80083FF02C0D4
:10EBF00081E008958091E80082FFF1CF06C0809106
:10EC0000F10081936150704031F08091F200909159
:10EC1000F300892BA1F78091E8008B778093E800BF
:10EC200061157105E1F605C08EB3882341F085308A
:10EC300041F08091E80080FFF7CF80E0089582E006
:10EC4000089583E008950F931F93DF93CF9300D02F
:10EC5000CDB7DEB7E2E9F1E08091F100819381E088
:10EC6000EA39F807C9F70BDD8091E80083FFE4C0BB
:10EC70008091920190919301953009F46DC0963086
:10EC800040F4913081F1913070F0933009F0D4C0AC
:10EC90002AC0983009F4A3C0993009F4B2C0963064
:10ECA00009F0CAC07CC0803809F4C6C0823809F0B7
:10ECB000C3C08091960187708093E9008091EB003A
:10ECC0001092E9002091E800277F2093E80090E06F
:10ECD00025E0969587952A95E1F781708093F1005C
:10ECE0001092F10087C0882319F0823009F0A4C087
:10ECF0008F71823009F0A0C080919401882331F592
:10ED000020919601277009F497C02093E900809123
:10ED1000EB0080FF1BC0933021F48091EB008062F8
:10ED200013C08091EB0080618093EB0081E090E064
:10ED300002C0880F991F2A95E2F78093EA0010928B
:10ED4000EA008091EB0088608093EB001092E9006C
:10ED50008091E800877F51C0882309F06DC0109131
:10ED600094011F770FB7F8948091E800877F809314
:10ED7000E800A0DD8091E80080FFFCCF8091E300F7
:10ED80008078812B8093E30080688093E3001123D7
:10ED900011F482E001C083E08EBB0FBF4DC08058EC
:10EDA000823008F049C08091940190919501609162
:10EDB0009601AE014F5F5F4F45DDBC01009709F43E
:10EDC0003BC08091E800877F8093E80089819A8129
:10EDD0009FDE8091E8008B778093E8002DC080381B
:10EDE00059F58091E800877F8093E8008091900139
:10EDF0008093F1008091E8008E778093E8005ADDDF
:10EE00001BC08823C9F4909194019230A8F480919A
:10EE1000E800877F8093E800909390014BDD80911C
:10EE20009001882331F48091E30087FD02C081E0E6
:10EE300001C084E08EBB53DC8091E80083FF0AC0F0
:10EE40008091EB0080628093EB008091E800877FE7
:10EE50008093E8000F900F90CF91DF911F910F9159
:10EE6000089508951F938EB3882361F01091E900EF
:10EE70001092E9008091E80083FF01C0E4DE177082
:10EE80001093E9001F910895F999FECF92BD81BDBD
:10EE9000F89A992780B50895262FF999FECF1FBAC1
:10EEA00092BD81BD20BD0FB6F894FA9AF99A0FBEB3
:08EEB00001960895F894FFCFCC
:10EEB8004C5546414344430001000000000000084F
:10EEC8001201100102000008EB034A2001000001B2
:10EED800000109023E00020100803209040000011D
:10EEE800020201000524001001042402040524067E
:10EEF8000001070582030800FF09040100020A0057
:10EF08000000070504021000010705830210000134
:10EF18000403090426034100560052002000430060
:10EF280044004300200042006F006F0074006C0032
:0CEF38006F0061006400650072000000C2
:10FFE0000C94C3F30C94D6F30C94E9F30C94FEF345
:0CFFF0000C9405F40C940CF40C9413F425
:040000031000E00009
:00000001FF
